S01100004D61696E626F6172642E7372656386
S11300000C943B000C9463000C9463000C94630008
S11300100C9463000C9463000C9463000C946300D0
S11300200C9463000C9463000C9463000C946300C0
S11300300C9463000C9463000C9463000C946300B0
S11300400C9463000C9463000C9463000C946300A0
S11300500C9463000C9463000C9463000C94630090
S11300600C9463000C9463000C9463000C94630080
S11300700C9463005E0211241FBECFEFD4E0DEBFF8
S1130080CDBF11E0A0E0B1E0EAEFF5E002C00590D9
S11300900D92A630B107D9F721E0A6E0B1E001C086
S11300A01D92AB30B207E1F710E0C6E7D0E004C020
S11300B02297FE010E94F702C437D107C9F70E94B4
S11300C009020C94FB020C940000FF920F931F93FF
S11300D0CF93DF931F92CDB7DEB7F82E092F162FDB
S11300E049830E94C40262E08F2D902F0E94E9028E
S11300F0612F8F2D902F0E94E9024981642F8F2D4B
S1130100902F0E94E9028F2D902F0F90DF91CF91B5
S11301101F910F91FF900C94C202CF93DF93D82FBD
S1130120C92F0E94C40260EC8D2F9C2F0E94E9020B
S11301308FE99FE00197F1F700C000008D2F9C2FFD
S11301400E94C2028FE39CE90197F1F700C000000E
S113015047E06AE28D2F9C2F0E94650040E969E226
S11301608D2F9C2F0E94650042E068E28D2F9C2F0A
S11301700E94650043E06BE28D2F9C2F0E94650076
S113018040E660E68D2F9C2F0E94650040E660E704
S11301908D2F9C2F0E94650040E060E28D2F9C2FE4
S11301A00E94650040E061E28D2F9C2F0E94650053
S11301B040E062E28D2F9C2F0E94650040E063E2E4
S11301C08D2F9C2F0E94650040E064E28D2F9C2FB0
S11301D00E94650040E065E28D2F9C2F0E9465001F
S11301E040E066E28D2F9C2F0E94650040E067E2AC
S11301F08D2F9C2F0E94650040E06CE08D2F9C2F7A
S1130200DF91CF910C946500FC014083518362839C
S11302100C948D00FF920F931F93CF93DF9300D024
S1130220CDB7DEB7F82E092F162F2A8349830E94F3
S1130230C40265E08F2D902F0E94E902612F8F2D5B
S1130240902F0E94E9024981642F8F2D902F0E94E4
S1130250E9022A81622F8F2D902F0E94E9028F2DAF
S1130260902F0F900F90DF91CF911F910F91FF90DE
S11302700C94C2021F93CF93DF93D82FC92F0E94EF
S1130280C40260EB8D2F9C2F0E94E9026FEF8D2F2B
S11302909C2F0E94E902182F6FEF8D2F9C2F0E9434
S11302A0E9028D2F9C2F0E94C202812FDF91CF91F2
S11302B01F9108959F92AF92BF92CF92DF92EF92D7
S11302C0FF920F931F93CF93DF931F92CDB7DEB7A7
S11302D05C016B010E943A01982E8983898186FD15
S11302E011C0898187FD7FC08FEF0F90DF91CF917F
S11302F01F910F91FF90EF90DF90CF90BF90AF9040
S11303009F900895C5010E94C40260E9C5010E943E
S1130310E9026FEFC5010E94E902282F30E0220FA5
S1130320331F220F331F220F331FF6013183208323
S11303306FEFC5010E94E902482F50E0569547959A
S1130340529542954F7045275F704527F6012081ED
S11303503181242B352B318320836FEFC5010E941B
S1130360E9026FEFC5010E94E9026FEFC5010E9427
S1130370E9028F70F60183838823A1F086010C5F64
S11303801F4F7601F5E0EF0EF11C8150E80EF11CD1
S11303906FEFC5010E94E902F80181938F01EE1508
S11303A0FF05B1F7C5010E94C202898183FD0EC019
S11303B0F6011282898120E086FF0FC041E06CE2E1
S11303C0C5010E940A01892D87708FCF81E0F60153
S11303D08283898120E086FDF1CF42E06CE2C50191
S11303E00E940A01F0CFC5010E94C40264E9C5015C
S11303F00E94E9028ECF84B1806E84B9089585B1DC
S11304008F7185B985B16295660F607E682B65B979
S11304100895CF93DF93CDB7DEB72C970FB6F8943A
S1130420DEBF0FBECDBF66E08AE091E00E94FF010F
S113043060E071E089E091E00E948A0283E291E049
S11304409A8389831B8282E08C838FEA8D838EEF6B
S11304508E830EC061E08AE091E00E94FF012FEFDD
S113046083ED90E3215080409040E1F700C000000C
S113047062E08AE091E00E94FF012FEF81EE94E0B8
S1130480215080409040E1F700C00000BE016F5F42
S11304907F4F86E091E00E945A018F3FD9F664E0D5
S11304A08AE091E00E94FF012FEF81EE94E0215059
S11304B080409040E1F700C00000DACFCF93DF9393
S11304C000D01F92CDB7DEB78AE091E00E94FB0115
S11304D089E091E00E947E0260E0CE0101960E94D4
S11304E0B90249815A816B8186E091E00E9404013E
S11304F00F900F900F90DF91CF91089586E0809335
S1130500CA00E9ECF0E080818860808387E680930C
S1130510CC000895FB019081992351F0319680918C
S1130520C80085FFFCCF9093CE0091919111F7CF35
S1130530089524B1266124B9239825B1217F25B9D2
S1130540DC011196ED91FC9112978081817F80836B
S11305502C9A0895CF93DF93EC010E94990288812D
S1130560811104C080E58CBD81E08DBDDF91CF9108
S1130570089521E0FC01208325E230E032832183C9
S11305800C94AA022C9A08952C98089598E080E07F
S113059060FD2A9A60FF2A98299866950000000059
S11305A00000000000000000000000000000000047
S11305B0000000000000000000000000299A000074
S11305C023B123FB222720F9880F822B915001F7B6
S11305D00895FC012081211106C06EBD0DB407FEF3
S11305E0FDCF8EB508950C94C602EE0FFF1F059043
S10D05F0F491E02D0994F894FFCF74
S10905FA626C610A0000BE
S9030000FC
